:020000040000FA
:0600000082EF08F012007F
:020006000000F8
:08000800D9CFE6FFE1CFD9FFDB
:10001000080EE126330EDF6EDE52320EDD6E280E44
:10002000F36E020EF3CFDBFF0C0EF36E030EF3CF75
:10003000DBFF010EF36E040EF3CFDBFF060EF36E53
:10004000050EF3CFDBFF060EDB6A070EDB6A0F013E
:100050003C6B966A3B6B0A0EE66E45EC08F0E55287
:10006000D9CF14F0DACF15F0070EDB500F011424AE
:10007000E96E000E1520EA6EEF5013E0D9CF14F0B0
:10008000DACF15F0070EDBCFF3FFDB2AF350142491
:10009000E96E000E1520EA6EEF50E66E0CD8E552C0
:1000A000DFD7080EE15C02E2E16AE552E16EE5525B
:1000B000E7CFD9FF1200D9CFE6FFE1CFD9FF849077
:1000C00084928494FE0EDB380F0B0F0BE66E25D85E
:1000D000E552FE0EDB500F0BE66E1FD8E55236D808
:1000E000E552E7CFD9FF1200D9CFE6FFE1CFD9FF24
:1000F000848084928494FE0EDB380F0B0F0BE66E27
:100100000CD8E552FE0EDB500F0BE66E06D8E5521A
:100110001DD8E552E7CFD9FF1200D9CFE6FFE1CFD6
:10012000D9FF800E9516FE0EDBCFE6FFF00E83148E
:10013000E552E710836E8484020EE66E9EEC08F0B2
:10014000E5528494E552E7CFD9FF1200D9CFE6FFFC
:10015000E1CFD9FF030EE1260F0E95128482849021
:100160008494848400008350100D010EF3CFDBFFD4
:100170008494848400000F0E8314DF6E8494010E37
:10018000DB50DF10E76E020EE7CFDBFF020EDBBEB7
:10019000E8D7030EE15C02E2E16AE552E16EE55266
:1001A000E7CFD9FF1200D9CFE6FFE1CFD9FFFE0E8E
:1001B000DBCFE6FF80DFE552FB0EDBCFF6FFFC0E68
:1001C000DBCFF7FFFD0EDBCFF8FF0800F55016E0A0
:1001D000D950FB0FE96EFF0EDA20EA6EEFCFF6FF83
:1001E000EE2AEFCFF7FF000EEE22EFCFF8FFEE2260
:1001F0000800F550E66E78DFE552DED7E552E7CF2E
:10020000D9FF1200D9CFE6FFE1CFD9FFFE0EDBCF39
:10021000E6FF51DFE552FC0EDBCFE9FFFD0EDBCF41
:10022000EAFFEF500EE0FC0EDBCFE9FFDB2AFD0E0C
:10023000DBCFEAFF01E3DB2AEF50E66E55DFE55244
:10024000EAD7E552E7CFD9FF1200D9CFE6FFE1CFD9
:10025000D9FFE652FC0EDBCFE6FF2DDFE552DF6A69
:10026000FB0EDB50DF5C0FE2FD0EDBCFE9FFDB2A8C
:10027000FE0EDBCFEAFF01E3DB2AEF50E66E34DF50
:10028000E552DF2AEDD7E552E552E7CFD9FF12005C
:10029000D9CFE6FFE1CFD9FFE652FE0EDBCFE6FF76
:1002A0000ADFE552DF6AFD0EDB50DF5C06E2200E5E
:1002B000E66E1ADFE552DF2AF6D7E552E552E7CFC0
:1002C000D9FF1200D9CFE6FFE1CFD9FFE652DF6AAE
:1002D000FC0EDB50DF5C12E2300E146EDF50E76E76
:1002E000FD0EDBCFE9FFFE0EDBCFEAFFE750E9268C
:1002F000000EEA221450EF26DF2AEAD7E552E55233
:10030000E7CFD9FF1200D9CFE6FFE1CFD9FFE65200
:10031000DF6AFC0EDB50DF5C12E20F0E146EDF5062
:10032000E76EFD0EDBCFE9FFFE0EDBCFEAFFE75005
:10033000E926000EEA221450EF16DF2AEAD7E5522A
:10034000E552E7CFD9FF1200D9CFE6FFE1CFD9FFC1
:100350000A0E146E14C00CF0FE0EDBCF07F090EC0A
:1003600008F00350300FE66E020EE76EFC0EDBCF96
:10037000E9FFFD0EDBCFEAFFE750E926000EEA2297
:10038000E552E750EF6E0A0E146E14C00CF0FE0E2C
:10039000DBCF07F090EC08F0FE0E07C0DBFF0A0E83
:1003A000146E14C00CF0FE0EDBCF07F090EC08F0DA
:1003B0000350300FE66E010EE76EFC0EDBCFE9FF57
:1003C000FD0EDBCFEAFFE750E926000EEA22E552F8
:1003D000E750EF6E0A0E146E14C00CF0FE0EDBCF69
:1003E00007F090EC08F00750300FE66EFC0EDBCF04
:1003F000E9FFFD0EDBCFEAFFE552E750EF6EE55275
:10040000E7CFD9FF1200D9CFE6FFE1CFD9FFE652FF
:10041000DF6A040EDF5C3EE2FD0EDBCF14F0FE0E61
:10042000DBCF15F00A0E0B6E0C6A14C006F015C077
:1004300007F05CEC08F002C014F003C015F0300EB9
:100440001426000E1522040ED880DF54E76EFB0E32
:10045000DBCFE9FFFC0EDBCFEAFFE750E926000E19
:10046000EA2214C0EFFF0A0E146E156AFD0EDBCFF0
:1004700006F0FE0EDBCF07F014C00BF015C00CF039
:100480005CEC08F0FD0E06C0DBFFFE0E07C0DBFFD4
:10049000DF2ABFD7300EE76EFD0EDBCF14F0FE0E65
:1004A000DBCF15F0E7501426000E1522FB0EDBCF34
:1004B000E9FFFC0EDBCFEAFF14C0EFFFE552E55287
:1004C000E7CFD9FF1200D9CFE6FFE1CFD9FFFD0E6C
:1004D000DBCFE9FFFE0EDBCFEAFFEF500F0B186E0C
:1004E000196A18BE1968640E1902F3CF19F01802C0
:1004F000F3CF18F0F4501926010EE76EFD0EDBCF96
:10050000E9FFFE0EDBCFEAFFE750E926000EEA2204
:10051000EF500F0B0A0DF3CF1AF01B6A1ABE1B68BF
:1005200018501A24166E19501B20176E020EE76E13
:10053000FD0EDBCFE9FFFE0EDBCFEAFFE750E92639
:10054000000EEA22EF500F0B1C6E1D6A1CBE1D68C8
:1005500016501C24146E17501D20156E14C0F3FF86
:1005600015C0F4FF00D0E552E7CFD9FF1200D9CF74
:10057000E6FFE1CFD9FFFD0EDBCFE9FFFE0EDBCFBB
:10058000EAFFEF500F0B1A6E1B6A1ABE1B68E80ECB
:100590001B02F3CF1BF0030E1A02F3501B26E80ECA
:1005A0001A02F3CF1AF0F4501B26010EE76EFD0E6F
:1005B000DBCFE9FFFE0EDBCFEAFFE750E926000EB6
:1005C000EA22EF500F0B640DF3CF1CF01D6A1CBE26
:1005D0001D681A501C24186E1B501D20196E020E27
:1005E000E76EFD0EDBCFE9FFFE0EDBCFEAFFE75043
:1005F000E926000EEA22EF500F0B0A0DF3CF1EF092
:100600001F6A1EBE1F6818501E24166E19501F2028
:10061000176E030EE76EFD0EDBCFE9FFFE0EDBCF9C
:10062000EAFFE750E926000EEA22EF500F0B206E9A
:10063000216A20BE216816502024146E17502120F4
:10064000156E14C0F3FF15C0F4FF00D0E552E7CFDC
:10065000D9FF1200D9CFE6FFE1CFD9FFFE0EDB387C
:100660000F0B3009E66EFC0EDBCFE9FFDB2AFD0E37
:10067000DBCFEAFF01E3DB2AE552E750EF6EFE0E27
:10068000DB500F0B3009E66EFC0EDBCFE9FFDB061B
:10069000FD0EDBCFEAFF01E2DB06E552E750EF6E2D
:1006A000E552E7CFD9FF12008ADAAEDC7C0E146E79
:1006B000100E156E166A14C0E6FF15C0E6FF16C0D0
:1006C000E6FF800EE66E6FDDE552E552E552E5523B
:1006D0006F0E146E100E156E166A14C0E6FF15C06C
:1006E000E6FF16C0E6FFC00EE66E5DDDE552E552A0
:1006F000E552E552E80EE66E45EC08F0E5525E0E76
:10070000146E100E156E166A14C0E6FF15C0E6FFD3
:1007100016C0E6FF800EE66E46DDE552E552E55274
:10072000E5524C0E146E100E156E166A14C0E6FFDC
:1007300015C0E6FF16C0E6FFC00EE66E34DDE552DA
:10074000E552E552E55281A0FED7D76AD66AD58E2A
:1007500081B0FED7D6CF68F0D7CF60F00001616BD3
:10076000626B636B080E1F0B60C014F061C015F064
:1007700062C016F063C017F007E0D8901436153643
:1007800016361736E806F9E168C018F0196A1A6AD1
:100790001B6A18AE03D019681A681B681450181029
:1007A0000001606F15501910616F16501A10626FBA
:1007B00017501B10636FD59E186A196AAA0E1A6E1D
:1007C000430E1B6E60C004F061C005F062C006F00D
:1007D00063C007F0E9EC05F005C01CF006C01DF091
:1007E00007C01EF008C01FF01CC00AF01DC00BF0AF
:1007F0001EC00CF01FC00DF018C005F019C006F0A7
:100800001AC007F01BC008F057EC06F005C014F042
:1008100006C015F007C016F008C017F00A6A240ECB
:100820000B6E740E0C6E490E0D6E14C005F015C0E3
:1008300006F016C007F017C008F004EC06F005C07B
:1008400064F006C065F007C066F008C067F0CD0E22
:100850000A6ECC0E0B6E0C6E3E0E0D6E64C005F073
:1008600065C006F066C007F067C008F0F3EC06F05C
:10087000010A05E17F0E806E818C818E818ACD0E0A
:100880000A6ECC0E0B6E0C6E3E0E0D6E64C005F043
:1008900065C006F066C007F067C008F0F3EC06F02C
:1008A000010A19E0CD0E0A6ECC0E0B6E4C0E0C6ECA
:1008B0003F0E0D6E64C005F065C006F066C007F01F
:1008C00067C008F0F3EC06F0010A05E17F0E806EC8
:1008D000818C819E818ACD0E0A6ECC0E0B6E4C0EE1
:1008E0000C6E3F0E0D6E64C005F065C006F066C06C
:1008F00007F067C008F0F3EC06F0010A18E09A0E62
:100900000A6E990E0B6E0C6E3F0E0D6E64C005F0F4
:1009100065C006F066C007F067C008F0F3EC06F0AB
:10092000010A05E17F0E806E819C819E818A9A0E6C
:100930000A6E990E0B6E0C6E3F0E0D6E64C005F0C4
:1009400065C006F066C007F067C008F0F3EC06F07B
:10095000010A18E0CD0E0A6ECC0E0B6E0C6E3F0E27
:100960000D6E64C005F065C006F066C007F067C094
:1009700008F0F3EC06F0010A05E17E0E806E819C22
:10098000819E818ACD0E0A6ECC0E0B6E0C6E3F0ED0
:100990000D6E64C005F065C006F066C007F067C064
:1009A00008F0F3EC06F0010A16E00A6A0B6A0C6A1A
:1009B000400E0D6E64C005F065C006F066C007F01D
:1009C00067C008F0F3EC06F0010A05E17C0E806ECA
:1009D000819C819E818A0A6A0B6A0C6A400E0D6EA8
:1009E00064C005F065C006F066C007F067C008F097
:1009F000F3EC06F0010A19E09A0E0A6E990E0B6EDE
:100A0000190E0C6E400E0D6E64C005F065C006F048
:100A100066C007F067C008F0F3EC06F0010A05E1D4
:100A2000780E806E819C819E818A9A0E0A6E990E44
:100A30000B6E190E0C6E400E0D6E64C005F065C095
:100A400006F066C007F067C008F0F3EC06F0010A94
:100A500017E0330E0A6E0B6E0C6E400E0D6E64C006
:100A600005F065C006F066C007F067C008F0F3EC5B
:100A700006F0010A05E1700E806E819C819E818ADC
:100A8000330E0A6E0B6E0C6E400E0D6E64C005F0D8
:100A900065C006F066C007F067C008F0F3EC06F02A
:100AA000010A19E0CD0E0A6ECC0E0B6E4C0E0C6EC8
:100AB000400E0D6E64C005F065C006F066C007F01C
:100AC00067C008F0F3EC06F0010A05E1600E806EE5
:100AD000819C819E818ACD0E0A6ECC0E0B6E4C0ECF
:100AE0000C6E400E0D6E64C005F065C006F066C069
:100AF00007F067C008F0F3EC06F0010A17E0660E95
:100B00000A6E0B6E0C6E400E0D6E64C005F065C073
:100B100006F066C007F067C008F0F3EC06F0010AC3
:100B200005E1400E806E819C819E818A660E0A6E70
:100B30000B6E0C6E400E0D6E64C005F065C006F0C5
:100B400066C007F067C008F0F3EC06F0010A04E0A5
:100B5000806A819C819E818A690EE66E000EE66E37
:100B60000A6A0B6AC80E0C6E420E0D6E64C005F068
:100B700065C006F066C007F067C008F057EC06F0E5
:100B8000C4EC06F006C014F007C015F014C0E6FF70
:100B900015C0E6FF38DCE552E552E552E552030E9A
:100BA000E66E8A0EE66E6A0EE66E000EE66E25ECC6
:100BB00001F0E552E552E552E552C5D51200010EAD
:100BC000936E0F01396BD56A946A3A6B926A386BEF
:020BD000120011
:0E0BD2000F9E0CD00F9E07AE09D0046C051EBE
:100BE000061E071EE86A0522062207220F8E07C08E
:100BF00001F006C000F005C013F004C012F09E0E14
:100C0000026E036A6DEF07F00F6AA9EC07F0C1EC02
:100C100007F00FB651EF07F00FA205D00FBA51EF52
:100C200007F058EF07F00FBA64EF07F00FA005D0F8
:100C30000FB851EF07F064EF07F00FB858EF07F067
:100C4000036A7F0E0824026EE86A03220D50025EDA
:100C5000E86A035A1A0E106E086A126A136A006A6A
:100C6000016A0A50055E0B50065A0C50075A000ED6
:100C7000085A09E70A5005260B5006220C50072295
:100C8000000E082201D0128AD890053606360736A3
:100C90000836D8901236133600360136102EE1D7BA
:100CA000075006100510D8A4128A6DEF07F00F6ADE
:100CB000A9EC07F0C1EC07F00FB651EF07F00FA257
:100CC00005D00FB851EF07F058EF07F00FAA05D085
:100CD0000FB051EF07F058EF07F00FB002D00FA898
:100CE00002D064EF07F0036A0D500824026EE86A30
:100CF00003227E0E025EE86A035A126A136A006AD1
:100D0000016A0C500702F4CF01F0F3CF00F00B5052
:100D10000702F3501326F4500022000E01220C505B
:100D20000602F3501326F4500022000E01220A504E
:100D30000702F3501226F4501322000E0022012263
:100D40000B500602F3501226F4501322000E00221C
:100D500001220C500502F3501226F4501322000E0B
:100D6000002201220A500602F4501226000E13221D
:100D7000002201220B500502F4501226000E13220D
:100D8000002201226DEF07F00F6AA9EC07F00FB601
:100D9000CEEF06F00FA20ED00FB405D07F0E076E77
:100DA000FF0E066E1FD0800E076E066A1BD0076A04
:100DB000066A18D00FB0FBD78F0E0860EDD77E0EF5
:100DC0000864F5D78E0E085C05E0D890073206322D
:100DD000082AF8D70FA406D0066C071EE86A072277
:100DE00007AEE5D71200FCEC06F00FB6000C0FB012
:100DF000000C0FA4000C010C0F6AA9EC07F0C1EC69
:100E000007F00FB612000FAE08D00FA004D00FA845
:100E100002D00F8012000F9012000D50085C0BE101
:100E20000C50075C08E10B50065C05E10A50055CBC
:100E300002E10F801200D8A002D00F8E10D008500F
:100E40000DC008F00D6E07500CC007F00C6E065078
:100E50000BC006F00B6E05500AC005F00A6E0D506F
:100E6000085C10E0FF0F09E00F900FB403D00FAE45
:100E70000F8412000FAE0F9412000D2AD8900C327E
:100E80000B320A320A50055E0B50065A0C50075AB4
:100E900007BEEAD7D890053606360736082EF8D7AB
:100EA000C8D77F0E086EFF0E076E066E056E120025
:100EB0007F0E0FBEFF0E086E02D07F0E086E800EF2
:100EC000076E066A056AF3D70FAE04D0800E086E6F
:100ED000076AF7D7086A076AF4D7015000101310A1
:100EE0001210F8E003BEF0D701BE0CD00250031080
:100EF000EBE0D89012361336003601360206D8A041
:100F00000306F2D70350D4E10228D2E012AE11D08A
:100F10007F0E121402E113A00CD0132AE86A0022FB
:100F2000012207E3D880013200321332022A02285C
:100F3000BFE00250C9E013C005F000C006F0013464
:100F4000076E0230086E0732089E0FBE088E57EFFC
:100F500007F00736083602E30F840F7E06E10F80A4
:100F6000086A076A066A056A1200082803E0D88042
:100F700007321200D890073202E10F8212000F866A
:100F800012000C360D3602E30F8C0F7E06E10F883F
:100F90000D6A0C6A0B6A0A6A12000D2803E0D880F9
:0E0FA0000C321200D8900C32EAE10F8A1200D7
:020FAE00060E2D
:100FB000F66E000EF76E000EF86E00010900F55097
:100FC000736F0900F550746F03E1736701D03DD072
:100FD0000900F5506E6F0900F5506F6F0900F5506C
:100FE000706F09000900F550E96E0900F550EA6ECE
:100FF000090009000900F550716F0900F550726F82
:1010000009000900F6CF75F0F7CF76F0F8CF77F04A
:101010006EC0F6FF6FC0F7FF70C0F8FF000171539C
:1010200002E1725307E00900F550EE6E7107F8E235
:101030007207F9D775C0F6FF76C0F7FF77C0F8FFE3
:0C10400000017307000E745BBFD71200A4
:04104C002020202020
:101050002020202020202020202020202000446943
:101060007374616E6365203D20202020636D004312
:10107000687269732026205A696164004465766548
:091080006C6F7065642062790058
:06108A00FF0EE350236E8F
:10109000EF0E01D0F30EE76EE72E4CEF08F00C0ECA
:1010A000226EE76AE72E52EF08F0222E51EF08F089
:0810B000232E4AEF08F01200A4
:0810B800036A026A100EE76EE4
:1010C000D89006360736023603360B50025C0C50B9
:1010D000035805E30B50025E0C50035A062AE72E14
:0410E000F0D7120033
:0C10E400000EF36E00EE00F0060E01D8C6
:1010F0001200EA6002D0EE6AFCD7F350E9601200F9
:04110000EE6AFCD7C0
:0C11040015EE00F025EE00F0F86A0F9CDC
:10111000D7EC07F0A9EC08F054EC03F0FBD7120071
:10112000036A080EE76ED890073603360C50035C4E
:0C11300002E3036E072AE72EF7D7120037
:04113C00FF0EE3506F
:10114000E84E1200000000D000D000D0E82EFAD700
:0211500012008B
:02115200120089
:00000001FF
